:03000000020200F9
:0400230002059B0037
:050030000000000000CB
:0400430002010000B6
:100100000202BA000200000002000000020000002B
:1001100002000000020000000200000002000000D7
:100120000200000002000000020485000204B90081
:1002000075815EE4F532F533F530F531F534C20031
:10021000C201A90074FE901000F0A3D9FC74FD90F7
:100220001100F0A3D9FC907F9474BFF0907F957477
:10023000EFF07410907F9EF07400907F98F07440FF
:10024000907F9DF07400907F97F07482907F9EF075
:10025000907F957403F0907FAFE0D2E0F07401904E
:100260007FABF0907FAEF0907FAC7404F0907FADE8
:100270007404F0907FC9F07407907FAFF074209001
:100280007F9CF07480907F98F07453F59875C83017
:100290007B059144D2CA759850D2E8D2AFD2AC74E3
:1002A00000F586907FD67402F0792E7A007B00DB11
:1002B000FEDAFAD9F67406F080FEC086C082C083EA
:1002C000C084C085C0E0E591C2E4F591907FAB7435
:1002D00001F0907FE8E0F9A3E0FAA3E0FBA3E0FCE3
:1002E000E95460B4000302035DB4406EBA000B121F
:1002F0000444400302042602042EBA010302042E21
:10030000BA020302042EBA0303020468BA041EBB35
:10031000000A907F95E04402F0020426907F98E066
:1003200054FDF0907F95E054FDF0020426BA0503D9
:1003300002042EBA0619BB0008E533D39532020435
:1003400002BB0108E532C3953302040202042EBA4F
:1003500007058B3402042602042E02042EBA002064
:10036000B98010907F00E4F0A3F0907FB57402F0A4
:10037000020426B9820280EBB9810280E602042ED3
:10038000BA010FBB000302042EBB010302042602C4
:10039000042EBA030FBB000302042EBB01030204A8
:1003A0002602042EBA0656BC010F907FD47406F0C4
:1003B000907FD5745AF0020426BC0212BB006F90E5
:1003C0007FD47406F0907FD5746CF0020426BC03D1
:1003D000297404C39B40576055EB2B90068C2582F3
:1003E000F58274003583F583E0F9A3E0FA907FD4B9
:1003F000E9F0907FD5EAF002042602042EBA080F35
:100400007401907F00F07401907FB5F0020426BA69
:100410000903020426BA0A057400020402BA0B0397
:1004200002042602042E907FB47402F08009907FAB
:10043000B4E04401F08000D0E0D085D084D083D0F7
:1004400082D08632EB20E71EC3940A5019EB232496
:1004500046F58274063400F583E0F5CBF5CDA3E0D4
:10046000F5CAF5CCC322D322B94111EB64FF548005
:10047000FB907F98E0547F4BF0020426907F9BE036
:1004800064FF020402C086C082C083C084C085C0ED
:10049000E0E591C2E4F591907FA97404F074209096
:1004A0007F9CF01205DC7420907F9CF0D0E0D0851A
:1004B000D084D083D082D08632C086C082C083C030
:1004C00084C085C0E07410907F9CF0E591C2E4F593
:1004D00091907FAA7404F0907FC9E0F9E4F58690CA
:1004E0007DC0758510853284E005860584F0E5843D
:1004F000B53302800905320586A3D9EC8000907FD0
:10050000C9F0B16D7420907F9CF0D0E0D085D0848C
:10051000D083D082D08632E4F586907FBCE020E1A3
:100520004B907D00E532F0A3E533F0A3E530F0A376
:10053000E531F0A3E430000104F0A305869010003B
:100540007910E0A30586F0A30586D9F6058674FC2C
:10055000F0A305869011007910E0A30586F0A305AD
:1005600086D9F6E4F586907FBD7426F0222000132C
:10057000E532B53301220533758310853382E0F50A
:1005800099D2007400B5340122E533D39532C39576
:100590003440F5753400D2010205DCC086C082C04B
:1005A00083C084C085C0E0309907C299C20012059B
:1005B000703098051205C6C298D0E0D085D084D09E
:1005C00083D082D086327583118530820582E59989
:1005D000F0E582B53101220530B1DC227410907F44
:1005E0009CF0907FB8E020E13E20013CE530B53141
:1005F0000122E4F5867583110586907E00F0A3053F
:10060000867901E530B5310280100531853182E00F
:100610000586F0A3058609B940E97410907F9CF027
:10062000907FB9E96001F022C201E4F586907E0076
:100630007401F0A37402F0907FB9F022C299F59989
:100640003099FDC29922E55EF63CFD8FFEC8FF643D
:10065000FFB2FFD9FFEDFFF3FFFA12010001FFFF28
:10066000FF40CD06040189AB01020301090220000D
:1006700001010080320904000002FFFFFF000705AE
:10068000820340000107050202400000069406981C
:1006900006BA06E8040300002203410043004D00AF
:1006A000450020007500730062002000770069009B
:1006B000640067006500740073002E03410043006E
:1006C0004D004500200055005300420020007300FB
:1006D00065007200690061006C002000770069000D
:0E06E0006400670065007400060334003700F4
:00000001FF
